:1000000012C02CC02BC02AC029C028C027C026C0BF
:1000100025C024C023C022C021C020C01FC01EC0D4
:100020001DC01CC01BC011241FBECFE5D4E0DEBF25
:10003000CDBF10E0A0E6B0E0E2EDFBE002C005902D
:100040000D92A236B107D9F710E0A2E6B0E001C0E8
:100050001D92A236B107E1F7DED4B9C5D1CFBF9268
:10006000CF92DF92DC01CB01B901E3E1FCE00F921A
:100070001F92D92EC82EBA2E242F172E062E099580
:100080001F900F90DF90CF90BF900895BF92CF92B6
:10009000DF92DC01CB01B901E3E9FFE00F921F928F
:1000A000D92EC82EBA2E242F172E062E09951F9052
:1000B0000F90DF90CF90BF900895CF93DF93DC0136
:1000C000CB01FA01E9012134310510F0C0E4D0E0A0
:1000D000AC01BD01407CCF019E0194D4CE01DF91E3
:1000E000CF9108952F923F924F925F926F927F929D
:1000F0008F929F92AF92BF92CF92DF92EF92FF9238
:100100000F931F93CF93DF93DC01CB01180189017B
:100110002134310510F000E410E028015694479492
:1001200030EC832E3FEF932E3FEFA32E3FEFB32E05
:1001300088229922AA22BB223A01DA0140E050E04B
:1001400030E020E019C0C401861997098A0F9B1F6F
:10015000FC01659174918D919D916817790709F063
:1001600021E080959095862B972B6FEF8F3F960718
:1001700009F031E04F5F5F4F4415550521F7222309
:1001800059F1332339F0C501B40143E020E030E0F8
:10019000F101099575016401C0E0D0E012C0D301FE
:1001A0002D913D913D01C701B60141E0F101099555
:1001B00082E090E0A0E0B0E0C80ED91EEA1EFB1E6F
:1001C0002196C415D50559F7C501B40145E020E0D5
:1001D00030E0F101099502C000E010E0C801DF91B4
:1001E000CF911F910F91FF90EF90DF90CF90BF9034
:1001F000AF909F908F907F906F905F904F903F90C7
:100200002F90089552C086C06BC06AC069C068C094
:1002100067C066C065C064C063C062C061C060C0C2
:100220005FC05EC05DC05CC05BC00000000000003D
:100230000000EC2DFD2DB7B6B0FCFDCF27BFE89533
:10024000B7B6B0FCFDCF21E1B7B6B6FCF4CF089548
:10025000FFFFFFFFFFFFFFFF090212000101008007
:100260003209040000000000000012011001FF002C
:100270000008C016DC050201010200010E03550052
:10028000530042006100730070001C037700770088
:1002900077002E00660069007300630068006C0040
:1002A0002E00640065000403090411241FBECFE57D
:1002B000D4E0DEBFCDBF10E0A0E6B0E0E8EFFFE1A4
:1002C00002C005900D92A836B107D9F710E0A8E654
:1002D000B0E001C01D92AE39B107E1F72FD18CC358
:1002E00091CFA82FB92F80E090E041E050EA6095CF
:1002F00030E009C02D9182279795879510F08427CB
:100300009527305EC8F36F5FA8F30895EADF8D93F9
:100310009D930895CF93CFB7CF93DF93C395869BDB
:10032000E9F7869B0BC0869B09C0869B07C0869B0E
:1003300005C0869B03C0869B01C089C06F93C09196
:100340008100DD27C857DF4F2F9365E5869B03C0EB
:100350002F916F91E6CF0F931F934F9320E040E1D1
:100360005F9300B3047406FB27F93F9350E03BE032
:1003700039C0147440642F77012F5F5F1EC040683E
:1003800010B314742F7752501FC0406400B32F77FE
:100390000474D1F15F5F00C023C0406210B32F77B7
:1003A000147491F15F5F00C025C004741027515090
:1003B00012F45D5F0000115027952C3F10B3C8F672
:1003C00014740127015027952C3FC8F64227499302
:1003D00000B3047410274F73115027952C3FA8F6D3
:1003E0004695469510B3147479F00127015027956E
:1003F0002C3F98F66B5A60F3315000B3B0F600C052
:1004000010E41ABF002717C03B503195C31BD040E2
:1004100010E41ABF0881033CF9F00B34E9F0209195
:100420007F001981110F1213EDCF093651F10D32F2
:1004300011F0013E39F7009386003F915F914F9193
:100440001F910F912F916F91CAB7C6FD67CFDF91B2
:10045000CF91CFBFCF91189520918600222369F3C9
:1004600010918400112339F534303AF1309384002F
:1004700020938000109181003BE0311B309381007C
:100480001CC0009184000130B4F40AE53091610091
:1004900034FD14C000936100C4E7D0E013C0052709
:1004A00010E000C0000002BB1AC0052710E0221FA8
:1004B0001DC010E021C04AE502C032ED432FC4E167
:1004C000D0E032E011B31464969A02B311BB54E445
:1004D00020E865E320FF052702BB279517951C3F01
:1004E000F0F66695B8F7B1F720FF052702BB279510
:1004F00017951C3FD0F62795179517FF0527000085
:100500001C3F02BBB0F629913A9519F70B7B10916D
:100510008500110FC651D04002BB11F010937F002F
:1005200010E41ABF006411B31B7B402F4B7B54E0D7
:100530005A95F1F702BB11BB42BB7FCF11BA80E8DD
:1005400082BB14BE81E08BBF82E08BBF879932C231
:1005500088E10FB6F89481BD11BC0FBE85B78260EB
:1005600085BF8BB780648BBF8E9A80E006C0EFE9B1
:10057000FFE03197F1F700C000008150C1F78E987D
:10058000789400918400035007FD7AC12091810086
:100590008CE090E0821B9109EC01C857DF4F20915D
:1005A00080002D3209F0E8C0083009F067C123EC63
:1005B000209374002AE5209361001092680048811E
:1005C000242F20763981222309F463C089E690E044
:1005D0009093830080938200333081F59B818C81DE
:1005E0002A81203339F48370E82FF0E0ED59FF4F72
:1005F000808120C0283529F4992371F4E1E0F0E0EE
:1006000006C0203571F49923A1F4E0E0F0E089E020
:100610008093570084910EC0983059F4E3E0F0E0E5
:10062000F6CF203A11F4D3D105C0203C11F46D81EE
:10063000D6D180E080936C0024E094C0353029F15D
:100640003A3019F1832F84508630A8F48A819B8137
:1006500090936E0080936D003930C9F02E81209305
:100660006F008D818270809370003093710047FD20
:1006700075C02FEF73C080916000323011F48E7F0F
:1006800001C081608093600002C021E06BC020E067
:1006900069C02A8110927D00332331F410927E00CC
:1006A0008DE790E022E055C0353019F420938500A5
:1006B00044C03630E1F5FC01E657FF4F20818557F5
:1006C0009F4FFC018081813019F486E698E104C0D7
:1006D000823041F484E598E1909383008093820016
:1006E00022E121C08330F1F4222341F482EA98E12F
:1006F000909383008093820024E015C0213041F460
:1007000086E898E190938300809382002CE10BC0EF
:10071000223041F488E798E190938300809382002F
:100720002EE001C020E080E4809368001BC03830D8
:1007300069F0393029F4209387008DE790E004C0F8
:100740008DE790E03A3021F020E003C087E890E0A8
:1007500021E0909383008093820004C080E880931E
:10076000680007C08F81882321F48E81821708F4E6
:10077000282F2093620082C08091680087FF7EC08E
:1007800080916F00801708F4082F801B80936F0002
:1007900011E0811110E080917100873008F466C08B
:1007A0007E010FC080916D0090916E009C012F5FC3
:1007B0003F4F30936E0020936D00F70161917F01F0
:1007C0000ED18E2D8C1B801768F354C080916D0064
:1007D00090916E0038E18030930708F04DC02E5F95
:1007E000F894E0916D00F0916E008991999131E05B
:1007F0000C0130935700E8951124789480916D0096
:1008000090916E00029690936E0080936D008F73AE
:100810009070009741F0112351F1201740F1809121
:100820007000882321F1F894E0916D00F0916E0042
:10083000329783E080935700E895789407B600FCE0
:10084000FDCFF894E0916D00F0916E00329785E055
:1008500080935700E895789407B600FCFDCFF89494
:1008600081E180935700E895789401C020E020173B
:1008700008F4ACCF112311F01092620010928400A2
:100880008091610084FF72C0809162008F3F09F403
:100890006DC0C82F893008F0C8E08C1B80936200BF
:1008A0008091740098E8892780937400CC2309F420
:1008B0004CC08091680087FF28C080916F008C1722
:1008C00008F4C82F8C1B80936F00D0E005E710E080
:1008D00019C080917100E0906D00F0906E0087303B
:1008E00018F0C70174D002C0F7018491F801808329
:1008F0000F5F1F4F0894E11CF11CF0926E00E09214
:100900006D00DF5FDC1729F71EC0E0918200F091D7
:10091000830086FF09C08C2FA5E7B0E094919D93DA
:1009200031968150D9F70BC0DF012C2F85E790E07D
:100930003D91FC013193CF01FD012150C9F7F093A6
:100940008300E0938200C93058F485E790E06C2F73
:10095000DDDCCC5FCC3041F08FEF8093620004C0CF
:100960008FEF80936200CEE1C093610084E190B389
:10097000947431F48150D9F71092850010927F0061
:1009800080916000803130F0879B0FC080916000C3
:10099000805109C0879909C080916000823028F099
:1009A0008091600082508093600080916000882375
:1009B00009F0E7CDF8948E9A12BA1BBE15BE81E0FD
:1009C0008BBF1BBEE0917200F09173000995E19915
:1009D000FECF9FBB8EBBE09A99278DB30895262F3B
:1009E000E199FECF9FBB8EBB2DBB0FB6F894E29A68
:1009F000E19A0FBE01960895F894FFCFFE5AFF1EAC
:100A000093070000FA01DC0102C005900D9221500D
:100A10003040D8F70895CF93DF93CDB7DEB7C054F9
:100A2000D0400FB6F894DEBF0FBECDBF88E10FB641
:100A3000F89481BD11BC0FBEF894198260916000DA
:100A40007091610020E030E0FB01E20FF31F45915F
:100A50005491F901E050F84E859194914817590747
:100A600019F081E0898306C02E5F3F4F88E0203077
:100A7000380751F78981882309F4A1C076E2C72E8F
:100A800078E1D72EE12CF12CC701B601AE014F5F02
:100A90005F4F20E430E011DB9C01C701B6016652D4
:100AA000794F8F4F9F4FAE014F5F5F4F0FE210E0C6
:100AB00019DB80E490E0A0E0B0E0C80ED91EEA1E89
:100AC000FB1E96E2C91699E1D90690E0E90690E08E
:100AD000F906D1F6C12C68E1D62EE12CF12CA12C1F
:100AE00058EEB52EAC0CBD1CCE0101966FEF70E038
:100AF00040E450E065D040916000509161004A0DA3
:100B00005B1D662757FD6095762FCE01019620E488
:100B100030E078DFC701B601AE014F5F5F4F20E4E0
:100B200030E006E410E0DEDA80E490E0A0E0B0E03F
:100B3000C80ED91EEA1EFB1E90E8C91699E1D90617
:100B400090E0E90690E0F90651F6C12C48E0D42E79
:100B5000CA18DB08CE0101966FEF70E040E450E068
:100B60002FD040916000509161004A0D5B1D6627B7
:100B700057FD6095762F9601A1E4CA16D10410F0B6
:100B800020E430E0CE0101963DDFB5016050784EA3
:100B900080E090E0AE014F5F5F4F20E430E00FE275
:100BA00010E0A0DA80E490E0A80EB91EA0ECBFEF40
:100BB000CA0EDB1EB0E0AB16B8E0BB0658F2FFCFA2
:100BC000DC0101C06D9341505040E0F70895F89466
:020BD000FFCF55
:020BD20004021B
:00000001FF
